:100000000C9446000C9463000C9463000C94630001
:100010000C9463000C9463000C9463000C946300D4
:100020000C9463000C9463000C9463000C946300C4
:100030000C9463000C9463000C9463000C946300B4
:100040000C94FC000C9463000C9463000C9463000B
:100050000C9463000C9463000C9463000C94630094
:100060000C9463000C9463000C9463000C94630084
:100070000C9463000C9463000C9463000C94630074
:100080000C9463000C9463000C94630011241FBE55
:10009000CFEFD0E1DEBFCDBF11E0A0E0B1E0EEE6F2
:1000A000F2E000E00BBF02C007900D92A030B10754
:1000B000D9F711E0A0E0B1E001C01D92A430B10772
:1000C000E1F70C9465000C940000CFEFD0E1DEBFA7
:1000D000CDBF0E94240180B7877F80BF80916400DC
:1000E000806180936400BC9A8091640088608093F2
:1000F000640000E010E080916500806180936500FD
:1001000080916500886080936500C49A0130110574
:1001100079F00230110524F40115110529F00FC002
:100120000230110559F00BC0809165008F7E03C02D
:1001300080916500877F8093650001C0C4980F5F40
:100140001F4F0330110514F000E010E0C3E6D0E0CB
:100150000E942B012197D7FFFBCFCDCF009731F025
:10016000A4E0B0E01197F1F70197D1F70895009757
:1001700031F0A0EABFE01197F1F70197D1F70895A8
:10018000CF93C82F882331F084E690E00E94AE0020
:10019000C150D1F7CF910895CF93C82F882331F064
:1001A0008AE090E00E94AE00C150D1F7CF9108954F
:1001B000CF93C82F882331F084E690E00E94B700E7
:1001C000C150D1F7CF910895CF93C82F882331F034
:1001D0008AE090E00E94B700C150D1F7CF91089516
:1001E000CF93C82F882331F081E090E00E94B700C0
:1001F000C150D1F7CF9108951F920F920FB60F9271
:1002000011248F939F938091020190910301019695
:1002100090930301809302010A976CF010920301FE
:10022000109202018091000190910101019690933A
:1002300001018093000186E082BF9F918F910F9012
:100240000FBE0F901F90189584E083BF12BE81E00F
:1002500087BF789408952091000130910101809129
:0E02600000019091010182179307C9F30895E0
:00000001FF
